:10000000E8C0000003C1000001C10000FFC0000003
:10001000FDC00000FBC00000F9C00000F7C00000F8
:10002000F5C00000F3C00000EEC100002CC20000CB
:10003000EDC00000EBC00000E9C00000E7C0000018
:10004000E5C00000E3C00000E1C00000DFC0000028
:10005000DDC00000DBC00000D9C00000D7C0000038
:10006000D5C00000D3C00000D1C00000CFC0000048
:10007000CDC00000CBC00000C9C00000C7C0000058
:10008000C5C00000C3C00000C1C00000BFC0000068
:10009000BDC00000BBC000004284A4830124C3048F
:1000A0000274A344C282E364D4430381231463949F
:1000B000B4C40A000A002064697400206461680006
:1000C0004368617220000A004F7070732C20756EB7
:1000D000737570706F7274656420636861726163B8
:1000E0007465723A200053706163650A00444F459D
:1000F0005320414E59424F4459205354494C4C20AF
:100100004B4E4F57204D4F52534520434F44453F90
:1001100000534F5300000100004C01120002000088
:100120005E01220022000080011500210000700104
:100130000900030000950104010309049901140258
:10014000030904AF0120000001C1260012010002D2
:1001500000000020C016790400010102000109021C
:100160002200010100C03209040000010300000068
:100170000921110100012215000705830320000158
:100180000631FF0974A1537508150026FF0095205C
:1001900009758102C004030904140359006F007536
:1001A00000720020004E0061006D0065000000201C
:1001B0000359006F00750072002000550053004283
:1001C00000200044006500760069006300650000BF
:1001D000000011241FBECFEFD0E2DEBFCDBF11E083
:1001E000A0E0B1E0E0E7F7E000E00BBF02C007905D
:1001F0000D92A030B107D9F711E0A0E0B1E001C045
:100200001D92A330B107E1F779D0B0C2F9CE0F93B8
:100210001F93CF93DF93182F803269F486EE90E01E
:1002200091D280EE95E120E931E0F9013197F1F7C3
:100230000197D9F74EC081548A3148F088EC90E09C
:1002400081D2812F9AD086EC90E07CD242C080ECA3
:1002500090E078D2812F91D08AE38FD0E12FF0E027
:10026000E95AFF4FE4910E2F07701E2FC0E9D1E02D
:1002700022C05E9A17FF0BC08BEB90E063D280E642
:1002800099E0FE013197F1F70197D9F70AC086EBA3
:1002900090E058D280E293E0FE013197F1F70197A8
:1002A000D9F75E9880E293E0FE013197F1F701976C
:1002B000D9F7110F01500023E1F684EB90E042D210
:1002C00080E496E020E931E0F9013197F1F70197F8
:1002D000D9F7DF91CF911F910F910895CF93DF93BD
:1002E000EC01FE0121968491882311F090DFF9CF73
:1002F00082EB90E027D2DF91CF9108951F93CF93A7
:10030000DF9380E88093610010926100569A5E98B6
:100310001DD010E0C0E9D1E00BC081E191E0DEDF4B
:1003200088E99AE3FE013197F1F70197D9F71F5F4A
:10033000163098F38DEE90E0D1DF80E49CE9FE0169
:100340003197F1F70197D9F710E0E7CF81E8809373
:10035000D70080EA8093D80086E189BD09B400FE09
:10036000FDCF80E98093D8001092E0001092000148
:100370008CE08093E20078940895482F80910001EA
:10038000882309F43EC02FB7F89483E08093E900F6
:1003900080910201882341F08091E80085FD02C030
:1003A0002FBF12C0109202019091E4009C5F33E0D5
:1003B0008091E80085FD13C02FBF8091E40089176C
:1003C00029F481E0809302018FEF0895809100016C
:1003D0008823B9F02FB7F8943093E900E9CF409320
:1003E000F1008091E80085FD06C08AE38093E80073
:1003F0001092010103C082E0809301012FBF80E0D1
:1004000008958FEF08951F920F920FB60F92112447
:100410008F939F938091E1001092E100982F83FFCA
:100420000FC01092E90081E08093EB001092EC0085
:1004300082E28093ED0088E08093F000109200014A
:1004400092FF1AC0809100018823B1F080910101D0
:10045000882391F0815080930101882369F483E01F
:100460008093E90002C01092F1008091E80085FDC0
:10047000FACF8AE38093E8009F918F910F900FBE8F
:100480000F901F9018951F920F920FB60F920BB6F8
:100490000F9211242F933F934F935F936F937F930A
:1004A0008F939F93AF93BF93CF93DF93EF93FF937C
:1004B0001092E9008091E80083FF2CC14091F10087
:1004C0003091F1008091F100A82FB0E02091F1006F
:1004D000922F80E0A82BB92B8091F100682F70E05B
:1004E0002091F100922F80E0682B792B8091F10010
:1004F000C82FD0E02091F100922F80E0C82BD92B9B
:1005000082EF8093E800363009F056C02CE131E0EC
:10051000A90145505040F9013797859194918A1768
:100520009B07E1F4FA018591949186179707B1F43E
:100530009A012E5F3F4FF901659174912E5F3F4FF5
:10054000F9012491CE01CF3FD10519F010F08FEFC2
:1005500090E0422F821758F4482F09C0295F3F4F7F
:10056000495F5F4FF1E02D343F07A9F6D3C05EEF3E
:100570008091E800282F30E0C90185709070892BA8
:10058000B9F322FDCAC0342F413208F030E2232FE4
:10059000CB0106C0FC010196E491E093F1002150EB
:1005A0002223C1F7630F711D431B5093E8004423BE
:1005B000F9F63032E9F2B1C0353061F48EEF809354
:1005C000E8008091E80080FFFCCF8A2F806880934C
:1005D000E300A3C0393031F5442309F09BC0A09358
:1005E00000018EEF8093E80086E491E021E0209303
:1005F000E900FC010196E491E093EB00EE2369F041
:10060000AC014F5F5F4FFC0184918093EC00CA0105
:100610000196FA0134913093ED002F5F253039F7C0
:100620008EE14DC0383061F4403809F073C08091DC
:10063000E80080FFFCCF809100018093F1001BC097
:100640003323E9F48091E80080FFFCCF423811F0B9
:1006500080E00DC06093E9008091EB0090E025E020
:10066000969587952A95E1F781701092E90080931D
:10067000F1001092F1008EEF8093E8004EC031300F
:1006800019F0333009F046C04230F1F4AB2BE1F4FD
:10069000262F2F77822F81508430B0F48EEF8093F5
:1006A000E8002093E9003330A9F189E18093EB0061
:1006B00081E090E002C0880F991F2A95E2F78093AD
:1006C000EA001092EA0029C0313021F5413A11F5D3
:1006D000672B01F54C2F5EEF8091E800282F30E06A
:1006E000C90185709070892BB9F322FD16C0942F33
:1006F000413208F090E2892F03C01092F10081503E
:100700008823D9F7491B5093E800442329F79032F6
:1007100019F303C081E28093EB00FF91EF91DF9129
:10072000CF91BF91AF919F918F917F916F915F9189
:100730004F913F912F910F900BBE0F900FBE0F90D6
:100740001F9018951F93CF93DF93EC01FE01219624
:100750001491112339F01A3011F48DE00EDE812F3F
:100760000CDEF4CFDF91CF911F910895F894FFCF65
:00000001FF
